 MFCN42D

 Timestamp is 35887162 (Wed Jun 17 18:46:10 1998)

 Preferred load address is 5f600000

 Start         Length     Name                   Class
 0001:00000000 00000cfeH .text                   CODE
 0001:00000d00 000003d7H .text$AFX_INIT          CODE
 0001:000010e0 00002243H .text$AFX_SOCK          CODE
 0001:00003330 00000203H .text$AFX_VDEL          CODE
 0001:00003540 000000d4H .text$x                 CODE
 0002:00000000 0000023cH .idata$5                DATA
 0002:00000240 000004dcH .rdata                  DATA
 0002:00000720 00000284H .rdata$r                DATA
 0002:000009a8 000001a0H .xdata$x                DATA
 0002:00000b48 00000020H .didat$2                DATA
 0002:00000b68 00000020H .didat$3                DATA
 0002:00000b88 00000070H .didat$4                DATA
 0002:00000bf8 00000070H .didat$7                DATA
 0002:00000c68 00000050H .idata$2                DATA
 0002:00000cb8 00000014H .idata$3                DATA
 0002:00000ccc 0000023cH .idata$4                DATA
 0002:00000f08 000001deH .idata$6                DATA
 0002:000010f0 000001ecH .edata                  DATA
 0003:00000000 00000004H .CRT$XCA                DATA
 0003:00000004 00000004H .CRT$XCL                DATA
 0003:00000008 00000004H .CRT$XCZ                DATA
 0003:0000000c 00000004H .CRT$XIA                DATA
 0003:00000010 00000004H .CRT$XIZ                DATA
 0003:00000020 000001a8H .data                   DATA
 0003:000001c8 00000070H .didat$5                DATA
 0003:00000238 00000058H .bss                    DATA
 0004:00000000 00000058H .rsrc$01                DATA
 0004:00000060 00000368H .rsrc$02                DATA

  Address         Publics by Value              Rva+Base     Lib:Object

 0001:00000000       ?GetHead@CSimpleList@@QBEPAXXZ 5f601000 f i dllnet.obj
 0001:00000010       ??1CNoTrackObject@@UAE@XZ  5f601010 f i sockcore.obj
 0001:00000030       ??_GCNoTrackObject@@UAEPAXI@Z 5f601030 f i sockcore.obj
 0001:00000030       ??_ECNoTrackObject@@UAEPAXI@Z 5f601030 f i sockcore.obj
 0001:00000060       ?T2A@@YAPADPAD@Z           5f601060 f i sockcore.obj
 0001:00000068       ?AfxGetModuleState@@YGPAVAFX_MODULE_STATE@@XZ 5f601068 f   MFC42D:MFC42D.DLL
 0001:0000006e       ?AfxTermThread@@YGXPAUHINSTANCE__@@@Z 5f60106e f   MFC42D:MFC42D.DLL
 0001:00000074       ?AfxTermExtensionModule@@YGXAAUAFX_EXTENSION_MODULE@@H@Z 5f601074 f   MFC42D:MFC42D.DLL
 0001:0000007a       ??0CDynLinkLibrary@@QAE@AAUAFX_EXTENSION_MODULE@@H@Z 5f60107a f   MFC42D:MFC42D.DLL
 0001:00000080       ??2CObject@@SGPAXI@Z       5f601080 f   MFC42D:MFC42D.DLL
 0001:00000086       ?AfxAssertFailedLine@@YGHPBDH@Z 5f601086 f   MFC42D:MFC42D.DLL
 0001:0000008c       ?AfxInitExtensionModule@@YGHAAUAFX_EXTENSION_MODULE@@PAUHINSTANCE__@@@Z 5f60108c f   MFC42D:MFC42D.DLL
 0001:00000092       ??3CObject@@SGXPAX@Z       5f601092 f   MFC42D:MFC42D.DLL
 0001:00000098       ?AfxGetAppModuleState@@YGPAVAFX_MODULE_STATE@@XZ 5f601098 f   MFC42D:MFC42D.DLL
 0001:0000009e       ??3@YAXPAX@Z               5f60109e f   MFC42D:MFC42D.DLL
 0001:000000a4       ??2@YAPAXI@Z               5f6010a4 f   MFC42D:MFC42D.DLL
 0001:000000aa       ??3CNoTrackObject@@SGXPAX@Z 5f6010aa f   MFC42D:MFC42D.DLL
 0001:000000b0       ?Serialize@CObject@@UAEXAAVCArchive@@@Z 5f6010b0 f   MFC42D:MFC42D.DLL
 0001:000000b6       ??0CObject@@IAE@XZ         5f6010b6 f   MFC42D:MFC42D.DLL
 0001:000000bc       ??4CString@@QAEABV0@PBD@Z  5f6010bc f   MFC42D:MFC42D.DLL
 0001:000000c2       ?AfxGetModuleThreadState@@YGPAVAFX_MODULE_THREAD_STATE@@XZ 5f6010c2 f   MFC42D:MFC42D.DLL
 0001:000000c8       ??1CObject@@UAE@XZ         5f6010c8 f   MFC42D:MFC42D.DLL
 0001:000000ce       ?GetValueAt@CMapPtrToPtr@@QBEPAXPAX@Z 5f6010ce f   MFC42D:MFC42D.DLL
 0001:000000d4       ??3CObject@@SGXPAXPBDH@Z   5f6010d4 f   MFC42D:MFC42D.DLL
 0001:000000da       ?Lookup@CMapPtrToPtr@@QBEHPAXAAPAX@Z 5f6010da f   MFC42D:MFC42D.DLL
 0001:000000e0       ?SetAt@CMapPtrToPtr@@QAEXPAX0@Z 5f6010e0 f   MFC42D:MFC42D.DLL
 0001:000000e6       ?FromHandlePermanent@CWnd@@SGPAV1@PAUHWND__@@@Z 5f6010e6 f   MFC42D:MFC42D.DLL
 0001:000000ec       ?AfxThrowResourceException@@YGXXZ 5f6010ec f   MFC42D:MFC42D.DLL
 0001:000000f2       ?AfxTrace@@YAXPBDZZ        5f6010f2 f   MFC42D:MFC42D.DLL
 0001:000000f8       ?CreateEx@CWnd@@QAEHKPBD0KHHHHPAUHWND__@@PAUHMENU__@@PAX@Z 5f6010f8 f   MFC42D:MFC42D.DLL
 0001:000000fe       ?AfxRegisterWndClass@@YGPBDIPAUHICON__@@PAUHBRUSH__@@0@Z 5f6010fe f   MFC42D:MFC42D.DLL
 0001:00000104       ??2CObject@@SGPAXIPBDH@Z   5f601104 f   MFC42D:MFC42D.DLL
 0001:0000010a       ?IsEmpty@CMapPtrToPtr@@QBEHXZ 5f60110a f   MFC42D:MFC42D.DLL
 0001:00000110       ?AfxEnableMemoryTracking@@YGHH@Z 5f601110 f   MFC42D:MFC42D.DLL
 0001:00000116       ?RemoveHead@CPtrList@@QAEPAXXZ 5f601116 f   MFC42D:MFC42D.DLL
 0001:0000011c       ?IsEmpty@CPtrList@@QBEHXZ  5f60111c f   MFC42D:MFC42D.DLL
 0001:00000122       ?RemoveAll@CMapPtrToPtr@@QAEXXZ 5f601122 f   MFC42D:MFC42D.DLL
 0001:00000128       ?AfxAssertValidObject@@YGXPBVCObject@@PBDH@Z 5f601128 f   MFC42D:MFC42D.DLL
 0001:0000012e       ?RemoveKey@CMapPtrToPtr@@QAEHPAX@Z 5f60112e f   MFC42D:MFC42D.DLL
 0001:00000134       ?AssertValid@CObject@@UBEXXZ 5f601134 f   MFC42D:MFC42D.DLL
 0001:0000013a       ??6CDumpContext@@QAEAAV0@I@Z 5f60113a f   MFC42D:MFC42D.DLL
 0001:00000140       ??6CDumpContext@@QAEAAV0@PBD@Z 5f601140 f   MFC42D:MFC42D.DLL
 0001:00000146       ?Dump@CObject@@UBEXAAVCDumpContext@@@Z 5f601146 f   MFC42D:MFC42D.DLL
 0001:0000014c       ?AddTail@CPtrList@@QAEPAU__POSITION@@PAX@Z 5f60114c f   MFC42D:MFC42D.DLL
 0001:00000152       ??2@YAPAXIPBDH@Z           5f601152 f   MFC42D:MFC42D.DLL
 0001:00000158       ?Delete@CException@@QAEXXZ 5f601158 f   MFC42D:MFC42D.DLL
 0001:0000015e       ?IsKindOf@CObject@@QBEHPBUCRuntimeClass@@@Z 5f60115e f   MFC42D:MFC42D.DLL
 0001:00000164       ?AfxGetThread@@YGPAVCWinThread@@XZ 5f601164 f   MFC42D:MFC42D.DLL
 0001:0000016a       ??6CDumpContext@@QAEAAV0@H@Z 5f60116a f   MFC42D:MFC42D.DLL
 0001:00000170       ??6CDumpContext@@QAEAAV0@PBX@Z 5f601170 f   MFC42D:MFC42D.DLL
 0001:00000176       ?GetBufferPtr@CFile@@UAEIIIPAPAX0@Z 5f601176 f   MFC42D:MFC42D.DLL
 0001:0000017c       ?SetFilePath@CFile@@UAEXPBD@Z 5f60117c f   MFC42D:MFC42D.DLL
 0001:00000182       ?GetFilePath@CFile@@UBE?AVCString@@XZ 5f601182 f   MFC42D:MFC42D.DLL
 0001:00000188       ?GetFileTitle@CFile@@UBE?AVCString@@XZ 5f601188 f   MFC42D:MFC42D.DLL
 0001:0000018e       ?GetFileName@CFile@@UBE?AVCString@@XZ 5f60118e f   MFC42D:MFC42D.DLL
 0001:00000194       ??1CFile@@UAE@XZ           5f601194 f   MFC42D:MFC42D.DLL
 0001:0000019a       ??0CFile@@QAE@XZ           5f60119a f   MFC42D:MFC42D.DLL
 0001:000001a0       ?AfxThrowFileException@@YGXHJPBD@Z 5f6011a0 f   MFC42D:MFC42D.DLL
 0001:000001a6       ?AfxThrowNotSupportedException@@YGXXZ 5f6011a6 f   MFC42D:MFC42D.DLL
 0001:000001ac       ?AssertValid@CFile@@UBEXXZ 5f6011ac f   MFC42D:MFC42D.DLL
 0001:000001b2       ??6CDumpContext@@QAEAAV0@PBVCObject@@@Z 5f6011b2 f   MFC42D:MFC42D.DLL
 0001:000001b8       ?GetDepth@CDumpContext@@QBEHXZ 5f6011b8 f   MFC42D:MFC42D.DLL
 0001:000001be       ?Dump@CFile@@UBEXAAVCDumpContext@@@Z 5f6011be f   MFC42D:MFC42D.DLL
 0001:000001c4       ?SetOccDialogInfo@CWnd@@MAEHPAU_AFX_OCC_DIALOG_INFO@@@Z 5f6011c4 f   MFC42D:MFC42D.DLL
 0001:000001ca       ?IsFrameWnd@CWnd@@UBEHXZ   5f6011ca f   MFC42D:MFC42D.DLL
 0001:000001d0       ?CheckAutoCenter@CWnd@@UAEHXZ 5f6011d0 f   MFC42D:MFC42D.DLL
 0001:000001d6       ?OnChildNotify@CWnd@@MAEHIIJPAJ@Z 5f6011d6 f   MFC42D:MFC42D.DLL
 0001:000001dc       ?PostNcDestroy@CWnd@@MAEXXZ 5f6011dc f   MFC42D:MFC42D.DLL
 0001:000001e2       ?DefWindowProcA@CWnd@@MAEJIIJ@Z 5f6011e2 f   MFC42D:MFC42D.DLL
 0001:000001e8       ?OnWndMsg@CWnd@@MAEHIIJPAJ@Z 5f6011e8 f   MFC42D:MFC42D.DLL
 0001:000001ee       ?WindowProc@CWnd@@MAEJIIJ@Z 5f6011ee f   MFC42D:MFC42D.DLL
 0001:000001f4       ?OnAmbientProperty@CWnd@@UAEHPAVCOleControlSite@@JPAUtagVARIANT@@@Z 5f6011f4 f   MFC42D:MFC42D.DLL
 0001:000001fa       ?PreTranslateMessage@CWnd@@UAEHPAUtagMSG@@@Z 5f6011fa f   MFC42D:MFC42D.DLL
 0001:00000200       ?EndModalState@CWnd@@UAEXXZ 5f601200 f   MFC42D:MFC42D.DLL
 0001:00000206       ?BeginModalState@CWnd@@UAEXXZ 5f601206 f   MFC42D:MFC42D.DLL
 0001:0000020c       ?DoDataExchange@CWnd@@MAEXPAVCDataExchange@@@Z 5f60120c f   MFC42D:MFC42D.DLL
 0001:00000212       ?GetSuperWndProcAddr@CWnd@@MAEPAP6GJPAUHWND__@@IIJ@ZXZ 5f601212 f   MFC42D:MFC42D.DLL
 0001:00000218       ?OnNotify@CWnd@@MAEHIJPAJ@Z 5f601218 f   MFC42D:MFC42D.DLL
 0001:0000021e       ?OnCommand@CWnd@@MAEHIJ@Z  5f60121e f   MFC42D:MFC42D.DLL
 0001:00000224       ?EndModalLoop@CWnd@@UAEXH@Z 5f601224 f   MFC42D:MFC42D.DLL
 0001:0000022a       ?ContinueModal@CWnd@@UAEHXZ 5f60122a f   MFC42D:MFC42D.DLL
 0001:00000230       ?WinHelpA@CWnd@@UAEXKI@Z   5f601230 f   MFC42D:MFC42D.DLL
 0001:00000236       ?GetScrollBarCtrl@CWnd@@UBEPAVCScrollBar@@H@Z 5f601236 f   MFC42D:MFC42D.DLL
 0001:0000023c       ?OnToolHitTest@CWnd@@UBEHVCPoint@@PAUtagTOOLINFOA@@@Z 5f60123c f   MFC42D:MFC42D.DLL
 0001:00000242       ?CalcWindowRect@CWnd@@UAEXPAUtagRECT@@I@Z 5f601242 f   MFC42D:MFC42D.DLL
 0001:00000248       ?PreCreateWindow@CWnd@@UAEHAAUtagCREATESTRUCTA@@@Z 5f601248 f   MFC42D:MFC42D.DLL
 0001:0000024e       ?DestroyWindow@CWnd@@UAEHXZ 5f60124e f   MFC42D:MFC42D.DLL
 0001:00000254       ?Create@CWnd@@UAEHPBD0KABUtagRECT@@PAV1@IPAUCCreateContext@@@Z 5f601254 f   MFC42D:MFC42D.DLL
 0001:0000025a       ?PreSubclassWindow@CWnd@@UAEXXZ 5f60125a f   MFC42D:MFC42D.DLL
 0001:00000260       ?GetConnectionHook@CCmdTarget@@MAEPAUIConnectionPoint@@ABU_GUID@@@Z 5f601260 f   MFC42D:MFC42D.DLL
 0001:00000266       ?GetExtraConnectionPoints@CCmdTarget@@MAEHPAVCPtrArray@@@Z 5f601266 f   MFC42D:MFC42D.DLL
 0001:0000026c       ?GetInterfaceHook@CCmdTarget@@UAEPAUIUnknown@@PBX@Z 5f60126c f   MFC42D:MFC42D.DLL
 0001:00000272       ?OnCreateAggregates@CCmdTarget@@UAEHXZ 5f601272 f   MFC42D:MFC42D.DLL
 0001:00000278       ?GetEventSinkMap@CCmdTarget@@MBEPBUAFX_EVENTSINKMAP@@XZ 5f601278 f   MFC42D:MFC42D.DLL
 0001:0000027e       ?GetInterfaceMap@CCmdTarget@@MBEPBUAFX_INTERFACEMAP@@XZ 5f60127e f   MFC42D:MFC42D.DLL
 0001:00000284       ?GetConnectionMap@CCmdTarget@@MBEPBUAFX_CONNECTIONMAP@@XZ 5f601284 f   MFC42D:MFC42D.DLL
 0001:0000028a       ?GetDispatchMap@CCmdTarget@@MBEPBUAFX_DISPMAP@@XZ 5f60128a f   MFC42D:MFC42D.DLL
 0001:00000290       ?GetCommandMap@CCmdTarget@@MBEPBUAFX_OLECMDMAP@@XZ 5f601290 f   MFC42D:MFC42D.DLL
 0001:00000296       ?GetTypeLib@CCmdTarget@@UAEJKPAPAUITypeLib@@@Z 5f601296 f   MFC42D:MFC42D.DLL
 0001:0000029c       ?GetTypeLibCache@CCmdTarget@@UAEPAVCTypeLibCache@@XZ 5f60129c f   MFC42D:MFC42D.DLL
 0001:000002a2       ?GetTypeInfoCount@CCmdTarget@@UAEIXZ 5f6012a2 f   MFC42D:MFC42D.DLL
 0001:000002a8       ?GetDispatchIID@CCmdTarget@@UAEHPAU_GUID@@@Z 5f6012a8 f   MFC42D:MFC42D.DLL
 0001:000002ae       ?IsInvokeAllowed@CCmdTarget@@UAEHJ@Z 5f6012ae f   MFC42D:MFC42D.DLL
 0001:000002b4       ?OnFinalRelease@CWnd@@UAEXXZ 5f6012b4 f   MFC42D:MFC42D.DLL
 0001:000002ba       ?OnCmdMsg@CCmdTarget@@UAEHIHPAXPAUAFX_CMDHANDLERINFO@@@Z 5f6012ba f   MFC42D:MFC42D.DLL
 0001:000002c0       ?Dump@CWnd@@UBEXAAVCDumpContext@@@Z 5f6012c0 f   MFC42D:MFC42D.DLL
 0001:000002c6       ?AssertValid@CWnd@@UBEXXZ  5f6012c6 f   MFC42D:MFC42D.DLL
 0001:000002cc       ?GetRuntimeClass@CWnd@@UBEPAUCRuntimeClass@@XZ 5f6012cc f   MFC42D:MFC42D.DLL
 0001:000002d2       ??0CWnd@@QAE@XZ            5f6012d2 f   MFC42D:MFC42D.DLL
 0001:000002d8       ??1CWnd@@UAE@XZ            5f6012d8 f   MFC42D:MFC42D.DLL
 0001:000002de       ??1CProcessLocalObject@@QAE@XZ 5f6012de f   MFC42D:MFC42D.DLL
 0001:000002e4       ?GetData@CProcessLocalObject@@QAEPAVCNoTrackObject@@P6GPAV2@XZ@Z 5f6012e4 f   MFC42D:MFC42D.DLL
 0001:000002ea       ??2CNoTrackObject@@SGPAXI@Z 5f6012ea f   MFC42D:MFC42D.DLL
 0001:000002f0       ___CxxFrameHandler         5f6012f0 f   msvcrtd:MSVCRTD.dll
 0001:00000300       ??_L@YGXPAXIHP6EX0@Z1@Z    5f601300 f   msvcrtd:ehvecctr.obj
 0001:000003a0       ??_M@YGXPAXIHP6EX0@Z@Z     5f6013a0 f   msvcrtd:ehvecdtr.obj
 0001:00000450       ?__ArrayUnwind@@YGXPAXIHP6EX0@Z@Z 5f601450 f   msvcrtd:ehvecdtr.obj
 0001:00000500       ??0type_info@@AAE@ABV0@@Z  5f601500 f   msvcrtd:ti_inst.obj
 0001:00000520       ??_Etype_info@@UAEPAXI@Z   5f601520 f i msvcrtd:ti_inst.obj
 0001:00000520       ??_Gtype_info@@UAEPAXI@Z   5f601520 f i msvcrtd:ti_inst.obj
 0001:00000550       ??4type_info@@AAEAAV0@ABV0@@Z 5f601550 f   msvcrtd:ti_inst.obj
 0001:00000560       _memset                    5f601560 f   msvcrtd:MSVCRTD.dll
 0001:00000570       __onexit                   5f601570 f   msvcrtd:atonexit.obj
 0001:000005b0       _atexit                    5f6015b0 f   msvcrtd:atonexit.obj
 0001:000005d0       __CRT_INIT@12              5f6015d0 f   msvcrtd:crtdll.obj
 0001:000006e0       __DllMainCRTStartup@12     5f6016e0 f   msvcrtd:crtdll.obj
 0001:000007d4       __except_handler3          5f6017d4 f   msvcrtd:MSVCRTD.dll
 0001:000007da       ?terminate@@YAXXZ          5f6017da f   msvcrtd:MSVCRTD.dll
 0001:000007e0       ??1type_info@@UAE@XZ       5f6017e0 f   msvcrtd:MSVCRTD.dll
 0001:000007e6       ___dllonexit               5f6017e6 f   msvcrtd:MSVCRTD.dll
 0001:000007ec       __free_dbg                 5f6017ec f   msvcrtd:MSVCRTD.dll
 0001:000007f2       __initterm                 5f6017f2 f   msvcrtd:MSVCRTD.dll
 0001:000007f8       __malloc_dbg               5f6017f8 f   msvcrtd:MSVCRTD.dll
 0001:000007fe       _FreeLibrary@4             5f6017fe f   kernel32:KERNEL32.dll
 0001:00000804       _GetModuleHandleA@4        5f601804 f   kernel32:KERNEL32.dll
 0001:0000080a       _LocalFree@4               5f60180a f   kernel32:KERNEL32.dll
 0001:00000810       _LocalAlloc@8              5f601810 f   kernel32:KERNEL32.dll
 0001:00000816       _LoadLibraryA@4            5f601816 f   kernel32:KERNEL32.dll
 0001:0000081c       _SetLastError@4            5f60181c f   kernel32:KERNEL32.dll
 0001:00000822       _PostMessageA@16           5f601822 f   user32:USER32.dll
 0001:00000828       _DispatchMessageA@4        5f601828 f   user32:USER32.dll
 0001:0000082e       _PeekMessageA@20           5f60182e f   user32:USER32.dll
 0001:00000834       _KillTimer@8               5f601834 f   user32:USER32.dll
 0001:0000083a       _WaitMessage@0             5f60183a f   user32:USER32.dll
 0001:00000840       _SetTimer@16               5f601840 f   user32:USER32.dll
 0001:00000846       __imp_load__WSACleanup@0   5f601846     wsock32:WSOCK32.dll
 0001:00000852       __tailMerge_WSOCK32        5f601852     wsock32:WSOCK32.dll
 0001:00000860       _WSACleanup@0              5f601860     wsock32:WSOCK32.dll
 0001:00000866       __imp_load__WSAStartup@8   5f601866     wsock32:WSOCK32.dll
 0001:00000872       _WSAStartup@8              5f601872     wsock32:WSOCK32.dll
 0001:00000878       __imp_load__WSASetLastError@4 5f601878     wsock32:WSOCK32.dll
 0001:00000884       _WSASetLastError@4         5f601884     wsock32:WSOCK32.dll
 0001:0000088a       __imp_load__inet_ntoa@4    5f60188a     wsock32:WSOCK32.dll
 0001:00000896       _inet_ntoa@4               5f601896     wsock32:WSOCK32.dll
 0001:0000089c       __imp_load__ntohs@4        5f60189c     wsock32:WSOCK32.dll
 0001:000008a8       _ntohs@4                   5f6018a8     wsock32:WSOCK32.dll
 0001:000008ae       __imp_load__accept@12      5f6018ae     wsock32:WSOCK32.dll
 0001:000008ba       _accept@12                 5f6018ba     wsock32:WSOCK32.dll
 0001:000008c0       __imp_load__htons@4        5f6018c0     wsock32:WSOCK32.dll
 0001:000008cc       _htons@4                   5f6018cc     wsock32:WSOCK32.dll
 0001:000008d2       __imp_load__inet_addr@4    5f6018d2     wsock32:WSOCK32.dll
 0001:000008de       _inet_addr@4               5f6018de     wsock32:WSOCK32.dll
 0001:000008e4       __imp_load__htonl@4        5f6018e4     wsock32:WSOCK32.dll
 0001:000008f0       _htonl@4                   5f6018f0     wsock32:WSOCK32.dll
 0001:000008f6       __imp_load__closesocket@4  5f6018f6     wsock32:WSOCK32.dll
 0001:00000902       _closesocket@4             5f601902     wsock32:WSOCK32.dll
 0001:00000908       __imp_load__gethostbyname@4 5f601908     wsock32:WSOCK32.dll
 0001:00000914       _gethostbyname@4           5f601914     wsock32:WSOCK32.dll
 0001:0000091a       __imp_load__recv@16        5f60191a     wsock32:WSOCK32.dll
 0001:00000926       _recv@16                   5f601926     wsock32:WSOCK32.dll
 0001:0000092c       __imp_load__send@16        5f60192c     wsock32:WSOCK32.dll
 0001:00000938       _send@16                   5f601938     wsock32:WSOCK32.dll
 0001:0000093e       __imp_load__WSAAsyncSelect@16 5f60193e     wsock32:WSOCK32.dll
 0001:0000094a       _WSAAsyncSelect@16         5f60194a     wsock32:WSOCK32.dll
 0001:00000950       __imp_load__WSAGetLastError@0 5f601950     wsock32:WSOCK32.dll
 0001:0000095c       _WSAGetLastError@0         5f60195c     wsock32:WSOCK32.dll
 0001:00000962       __imp_load__socket@12      5f601962     wsock32:WSOCK32.dll
 0001:0000096e       _socket@12                 5f60196e     wsock32:WSOCK32.dll
 0001:00000974       __imp_load__recvfrom@24    5f601974     wsock32:WSOCK32.dll
 0001:00000980       _recvfrom@24               5f601980     wsock32:WSOCK32.dll
 0001:00000986       __imp_load__sendto@24      5f601986     wsock32:WSOCK32.dll
 0001:00000992       _sendto@24                 5f601992     wsock32:WSOCK32.dll
 0001:00000998       __imp_load__connect@12     5f601998     wsock32:WSOCK32.dll
 0001:000009a4       _connect@12                5f6019a4     wsock32:WSOCK32.dll
 0001:000009aa       __imp_load__getpeername@12 5f6019aa     wsock32:WSOCK32.dll
 0001:000009b6       _getpeername@12            5f6019b6     wsock32:WSOCK32.dll
 0001:000009bc       __imp_load__getsockname@12 5f6019bc     wsock32:WSOCK32.dll
 0001:000009c8       _getsockname@12            5f6019c8     wsock32:WSOCK32.dll
 0001:000009ce       __imp_load__setsockopt@20  5f6019ce     wsock32:WSOCK32.dll
 0001:000009da       _setsockopt@20             5f6019da     wsock32:WSOCK32.dll
 0001:000009e0       __imp_load__getsockopt@20  5f6019e0     wsock32:WSOCK32.dll
 0001:000009ec       _getsockopt@20             5f6019ec     wsock32:WSOCK32.dll
 0001:000009f2       __imp_load__bind@12        5f6019f2     wsock32:WSOCK32.dll
 0001:000009fe       _bind@12                   5f6019fe     wsock32:WSOCK32.dll
 0001:00000a04       __imp_load__ioctlsocket@12 5f601a04     wsock32:WSOCK32.dll
 0001:00000a10       _ioctlsocket@12            5f601a10     wsock32:WSOCK32.dll
 0001:00000a16       __imp_load__listen@8       5f601a16     wsock32:WSOCK32.dll
 0001:00000a22       _listen@8                  5f601a22     wsock32:WSOCK32.dll
 0001:00000a28       __imp_load__shutdown@8     5f601a28     wsock32:WSOCK32.dll
 0001:00000a34       _shutdown@8                5f601a34     wsock32:WSOCK32.dll
 0001:00000a3a       ___delayLoadHelper@8       5f601a3a f   delayimp:delayhlp.obj
 0001:00000c33       ___FUnloadDelayLoadedDLL@4 5f601c33 f   delayimp:delayhlp.obj
 0001:00000ce6       _GetProcAddress@8          5f601ce6 f   kernel32:KERNEL32.dll
 0001:00000cec       _InterlockedExchange@8     5f601cec f   kernel32:KERNEL32.dll
 0001:00000cf2       _RaiseException@16         5f601cf2 f   kernel32:KERNEL32.dll
 0001:00000cf8       _GetLastError@0            5f601cf8 f   kernel32:KERNEL32.dll
 0001:00000d00       _RawDllMain@12             5f601d00 f   dllnet.obj
 0001:00000d9e       _DllMain@12                5f601d9e f   dllnet.obj
 0001:00000e5d       ?AfxNetInitModule@@YGXXZ   5f601e5d f   dllnet.obj
 0001:00000f20       ?_GetBaseClass@CAsyncSocket@@KGPAUCRuntimeClass@@XZ 5f601f20 f   sockcore.obj
 0001:00000f2a       ?GetRuntimeClass@CAsyncSocket@@UBEPAUCRuntimeClass@@XZ 5f601f2a f   sockcore.obj
 0001:00000f3a       ?_GetBaseClass@CSocket@@KGPAUCRuntimeClass@@XZ 5f601f3a f   sockcore.obj
 0001:00000f44       ?GetRuntimeClass@CSocket@@UBEPAUCRuntimeClass@@XZ 5f601f44 f   sockcore.obj
 0001:00000f54       ?_GetBaseClass@CSocketFile@@KGPAUCRuntimeClass@@XZ 5f601f54 f   sockcore.obj
 0001:00000f5e       ?GetRuntimeClass@CSocketFile@@UBEPAUCRuntimeClass@@XZ 5f601f5e f   sockcore.obj
 0001:00000fb0       ??1?$CProcessLocal@V_AFX_SOCK_STATE@@@@QAE@XZ 5f601fb0 f i sockcore.obj
 0001:00000fd0       ??C?$CEmbeddedButActsLikePtr@VCMapPtrToPtr@@@@QAEPAVCMapPtrToPtr@@XZ 5f601fd0 f i sockcore.obj
 0001:00000fd0       ??C?$CEmbeddedButActsLikePtr@VCPtrList@@@@QAEPAVCPtrList@@XZ 5f601fd0 f i sockcore.obj
 0001:00000fe0       ?GetData@?$CProcessLocal@V_AFX_SOCK_STATE@@@@QAEPAV_AFX_SOCK_STATE@@XZ 5f601fe0 f i sockcore.obj
 0001:00001030       ?CreateObject@?$CProcessLocal@V_AFX_SOCK_STATE@@@@SGPAVCNoTrackObject@@XZ 5f602030 f i sockcore.obj
 0001:000010a0       ??0_AFX_SOCK_STATE@@QAE@XZ 5f6020a0 f i sockcore.obj
 0001:000010c0       ??0CNoTrackObject@@QAE@XZ  5f6020c0 f i sockcore.obj
 0001:000010e0       ??1_AFX_SOCK_STATE@@UAE@XZ 5f6020e0 f   sockcore.obj
 0001:00001138       ?AfxSocketTerm@@YGXXZ      5f602138 f   sockcore.obj
 0001:0000117b       ?AfxSocketInit@@YGHPAUWSAData@@@Z 5f60217b f   sockcore.obj
 0001:0000121c       ??0CAsyncSocket@@QAE@XZ    5f60221c f   sockcore.obj
 0001:00001245       ?Create@CAsyncSocket@@QAEHIHJPBD@Z 5f602245 f   sockcore.obj
 0001:000012a5       ?Attach@CAsyncSocket@@QAEHIJ@Z 5f6022a5 f   sockcore.obj
 0001:000012f9       ?Detach@CAsyncSocket@@QAEIXZ 5f6022f9 f   sockcore.obj
 0001:0000133c       ?GetPeerName@CAsyncSocket@@QAEHAAVCString@@AAI@Z 5f60233c f   sockcore.obj
 0001:000013a4       ?GetSockName@CAsyncSocket@@QAEHAAVCString@@AAI@Z 5f6023a4 f   sockcore.obj
 0001:0000140c       ?Accept@CAsyncSocket@@UAEHAAV1@PAUsockaddr@@PAH@Z 5f60240c f   sockcore.obj
 0001:000014f4       ?Bind@CAsyncSocket@@QAEHIPBD@Z 5f6024f4 f   sockcore.obj
 0001:00001598       ?Close@CAsyncSocket@@UAEXXZ 5f602598 f   sockcore.obj
 0001:000015f7       ?Connect@CAsyncSocket@@QAEHPBDI@Z 5f6025f7 f   sockcore.obj
 0001:000016ca       ?Receive@CAsyncSocket@@UAEHPAXHH@Z 5f6026ca f   sockcore.obj
 0001:000016ef       ?ReceiveFrom@CAsyncSocket@@QAEHPAXHAAVCString@@AAIH@Z 5f6026ef f   sockcore.obj
 0001:00001763       ?Send@CAsyncSocket@@UAEHPBXHH@Z 5f602763 f   sockcore.obj
 0001:00001788       ?SendTo@CAsyncSocket@@QAEHPBXHIPBDH@Z 5f602788 f   sockcore.obj
 0001:00001854       ?AsyncSelect@CAsyncSocket@@QAEHJ@Z 5f602854 f   sockcore.obj
 0001:000018dd       ?OnReceive@CAsyncSocket@@MAEXH@Z 5f6028dd f   sockcore.obj
 0001:000018ea       ?OnSend@CAsyncSocket@@MAEXH@Z 5f6028ea f   sockcore.obj
 0001:000018f7       ?OnOutOfBandData@CAsyncSocket@@MAEXH@Z 5f6028f7 f   sockcore.obj
 0001:00001904       ?OnAccept@CAsyncSocket@@MAEXH@Z 5f602904 f   sockcore.obj
 0001:00001911       ?OnConnect@CAsyncSocket@@MAEXH@Z 5f602911 f   sockcore.obj
 0001:0000191e       ?OnClose@CAsyncSocket@@MAEXH@Z 5f60291e f   sockcore.obj
 0001:0000192b       ??1CAsyncSocket@@UAE@XZ    5f60292b f   sockcore.obj
 0001:00001985       ?LookupHandle@CAsyncSocket@@SGPAV1@IH@Z 5f602985 f   sockcore.obj
 0001:000019eb       ?AttachHandle@CAsyncSocket@@SGXIPAV1@H@Z 5f6029eb f   sockcore.obj
 0001:00001c33       ?DetachHandle@CAsyncSocket@@SGXIH@Z 5f602c33 f   sockcore.obj
 0001:00001de3       ?KillSocket@CAsyncSocket@@SGXIPAV1@@Z 5f602de3 f   sockcore.obj
 0001:00001e5f       ?DoCallBack@CAsyncSocket@@SGXIJ@Z 5f602e5f f   sockcore.obj
 0001:0000200d       ?Socket@CAsyncSocket@@QAEHHJHH@Z 5f60300d f   sockcore.obj
 0001:00002085       ?AssertValid@CAsyncSocket@@UBEXXZ 5f603085 f   sockcore.obj
 0001:000020d1       ?Dump@CAsyncSocket@@UBEXAAVCDumpContext@@@Z 5f6030d1 f   sockcore.obj
 0001:0000212a       ?ReceiveFromHelper@CAsyncSocket@@MAEHPAXHPAUsockaddr@@PAHH@Z 5f60312a f   sockcore.obj
 0001:00002157       ?SendToHelper@CAsyncSocket@@MAEHPBXHPBUsockaddr@@HH@Z 5f603157 f   sockcore.obj
 0001:00002184       ?ConnectHelper@CAsyncSocket@@MAEHPBUsockaddr@@H@Z 5f603184 f   sockcore.obj
 0001:000021af       ??0CSocket@@QAE@XZ         5f6031af f   sockcore.obj
 0001:000021ec       ?CancelBlockingCall@CSocket@@QAEXXZ 5f6031ec f   sockcore.obj
 0001:00002216       ?OnMessagePending@CSocket@@MAEHXZ 5f603216 f   sockcore.obj
 0001:00002249       ??1CSocket@@UAE@XZ         5f603249 f   sockcore.obj
 0001:000022a3       ?Accept@CSocket@@UAEHAAVCAsyncSocket@@PAUsockaddr@@PAH@Z 5f6032a3 f   sockcore.obj
 0001:0000230d       ?Close@CSocket@@UAEXXZ     5f60330d f   sockcore.obj
 0001:00002369       ?Receive@CSocket@@UAEHPAXHH@Z 5f603369 f   sockcore.obj
 0001:000023da       ?Send@CSocket@@UAEHPBXHH@Z 5f6033da f   sockcore.obj
 0001:0000244e       ?SendChunk@CSocket@@QAEHPBXHH@Z 5f60344e f   sockcore.obj
 0001:000024a8       ?ConnectHelper@CSocket@@MAEHPBUsockaddr@@H@Z 5f6034a8 f   sockcore.obj
 0001:00002537       ?ReceiveFromHelper@CSocket@@MAEHPAXHPAUsockaddr@@PAHH@Z 5f603537 f   sockcore.obj
 0001:000025b0       ?SendToHelper@CSocket@@MAEHPBXHPBUsockaddr@@HH@Z 5f6035b0 f   sockcore.obj
 0001:0000262a       ?ProcessAuxQueue@CSocket@@SGHXZ 5f60362a f   sockcore.obj
 0001:00002733       ?AuxQueueAdd@CSocket@@KGXIIJ@Z 5f603733 f   sockcore.obj
 0001:00002795       ?PumpMessages@CSocket@@MAEHI@Z 5f603795 f   sockcore.obj
 0001:00002a55       ?AssertValid@CSocket@@MBEXXZ 5f603a55 f   sockcore.obj
 0001:00002a68       ?Dump@CSocket@@MBEXAAVCDumpContext@@@Z 5f603a68 f   sockcore.obj
 0001:00002acf       ??0CSocketFile@@QAE@PAVCSocket@@H@Z 5f603acf f   sockcore.obj
 0001:00002be9       ??1CSocketFile@@UAE@XZ     5f603be9 f   sockcore.obj
 0001:00002c05       ?Read@CSocketFile@@UAEIPAXI@Z 5f603c05 f   sockcore.obj
 0001:00002d4a       ?Write@CSocketFile@@UAEXPBXI@Z 5f603d4a f   sockcore.obj
 0001:00002dbb       ?Close@CSocketFile@@UAEXXZ 5f603dbb f   sockcore.obj
 0001:00002dd0       ?Open@CSocketFile@@UAEHPBDIPAVCFileException@@@Z 5f603dd0 f   sockcore.obj
 0001:00002de4       ?Duplicate@CSocketFile@@UBEPAVCFile@@XZ 5f603de4 f   sockcore.obj
 0001:00002df6       ?GetPosition@CSocketFile@@UBEKXZ 5f603df6 f   sockcore.obj
 0001:00002e08       ?Seek@CSocketFile@@UAEJJI@Z 5f603e08 f   sockcore.obj
 0001:00002e35       ?SetLength@CSocketFile@@UAEXK@Z 5f603e35 f   sockcore.obj
 0001:00002e47       ?GetLength@CSocketFile@@UBEKXZ 5f603e47 f   sockcore.obj
 0001:00002e59       ?LockRange@CSocketFile@@UAEXKK@Z 5f603e59 f   sockcore.obj
 0001:00002e6b       ?UnlockRange@CSocketFile@@UAEXKK@Z 5f603e6b f   sockcore.obj
 0001:00002e7d       ?Flush@CSocketFile@@UAEXXZ 5f603e7d f   sockcore.obj
 0001:00002e88       ?Abort@CSocketFile@@UAEXXZ 5f603e88 f   sockcore.obj
 0001:00002e98       ?AssertValid@CSocketFile@@UBEXXZ 5f603e98 f   sockcore.obj
 0001:00002eca       ?Dump@CSocketFile@@UBEXAAVCDumpContext@@@Z 5f603eca f   sockcore.obj
 0001:00002f22       ??0CSocketWnd@@QAE@XZ      5f603f22 f   sockcore.obj
 0001:00002f41       ?OnSocketNotify@CSocketWnd@@IAEJIJ@Z 5f603f41 f   sockcore.obj
 0001:00002f67       ?OnSocketDead@CSocketWnd@@IAEJIJ@Z 5f603f67 f   sockcore.obj
 0001:00002f8d       ?_GetBaseMessageMap@CSocketWnd@@KGPBUAFX_MSGMAP@@XZ 5f603f8d f   sockcore.obj
 0001:00002f97       ?GetMessageMap@CSocketWnd@@MBEPBUAFX_MSGMAP@@XZ 5f603f97 f   sockcore.obj
 0001:00002fa7       ??BCAsyncSocket@@QBEIXZ    5f603fa7 f   sockcore.obj
 0001:00002fb8       ?GetPeerName@CAsyncSocket@@QAEHPAUsockaddr@@PAH@Z 5f603fb8 f   sockcore.obj
 0001:00002fe3       ?GetSockName@CAsyncSocket@@QAEHPAUsockaddr@@PAH@Z 5f603fe3 f   sockcore.obj
 0001:0000300e       ?SetSockOpt@CAsyncSocket@@QAEHHPBXHH@Z 5f60400e f   sockcore.obj
 0001:00003041       ?GetSockOpt@CAsyncSocket@@QAEHHPAXPAHH@Z 5f604041 f   sockcore.obj
 0001:00003074       ?FromHandle@CAsyncSocket@@SGPAV1@I@Z 5f604074 f   sockcore.obj
 0001:00003086       ?GetLastError@CAsyncSocket@@SGHXZ 5f604086 f   sockcore.obj
 0001:00003090       ?Bind@CAsyncSocket@@QAEHPBUsockaddr@@H@Z 5f604090 f   sockcore.obj
 0001:000030bb       ?Connect@CAsyncSocket@@QAEHPBUsockaddr@@H@Z 5f6040bb f   sockcore.obj
 0001:000030db       ?IOCtl@CAsyncSocket@@QAEHJPAK@Z 5f6040db f   sockcore.obj
 0001:00003106       ?Listen@CAsyncSocket@@QAEHH@Z 5f604106 f   sockcore.obj
 0001:0000312d       ?ReceiveFrom@CAsyncSocket@@QAEHPAXHPAUsockaddr@@PAHH@Z 5f60412d f   sockcore.obj
 0001:00003159       ?ShutDown@CAsyncSocket@@QAEHH@Z 5f604159 f   sockcore.obj
 0001:00003180       ?SendTo@CAsyncSocket@@QAEHPBXHPBUsockaddr@@HH@Z 5f604180 f   sockcore.obj
 0001:000031ac       ?Create@CSocket@@QAEHIHPBD@Z 5f6041ac f   sockcore.obj
 0001:000031cf       ?IsBlocking@CSocket@@QAEHXZ 5f6041cf f   sockcore.obj
 0001:000031e8       ?FromHandle@CSocket@@SGPAV1@I@Z 5f6041e8 f   sockcore.obj
 0001:000031fa       ?Attach@CSocket@@QAEHI@Z   5f6041fa f   sockcore.obj
 0001:00003220       ??_E_AFX_SOCK_STATE@@UAEPAXI@Z 5f604220 f i sockcore.obj
 0001:00003220       ??_G_AFX_SOCK_STATE@@UAEPAXI@Z 5f604220 f i sockcore.obj
 0001:00003250       ??_GCAsyncSocket@@UAEPAXI@Z 5f604250 f i sockcore.obj
 0001:00003280       ??_GCSocket@@UAEPAXI@Z     5f604280 f i sockcore.obj
 0001:000032b0       ??_ECSocketFile@@UAEPAXI@Z 5f6042b0 f i sockcore.obj
 0001:000032b0       ??_GCSocketFile@@UAEPAXI@Z 5f6042b0 f i sockcore.obj
 0001:000032e0       ??_ECSocketWnd@@UAEPAXI@Z  5f6042e0 f i sockcore.obj
 0001:000032e0       ??_GCSocketWnd@@UAEPAXI@Z  5f6042e0 f i sockcore.obj
 0001:00003310       ??1CSocketWnd@@UAE@XZ      5f604310 f i sockcore.obj
 0001:00003440       ??_ECAsyncSocket@@UAEPAXI@Z 5f604440 f i dllnet.obj
 0001:000034b0       ??_ECSocket@@UAEPAXI@Z     5f6044b0 f i dllnet.obj
 0001:00003520       ??B?$CTypedSimpleList@PAUCRuntimeClass@@@@QAEPAUCRuntimeClass@@XZ 5f604520 f i dllnet.obj
 0001:00003520       ??B?$CTypedSimpleList@PAVCOleObjectFactory@@@@QAEPAVCOleObjectFactory@@XZ 5f604520 f i dllnet.obj
 0002:00000000       __imp__FreeLibrary@4       5f605000     kernel32:KERNEL32.dll
 0002:00000004       __imp__GetModuleHandleA@4  5f605004     kernel32:KERNEL32.dll
 0002:00000008       __imp__LocalFree@4         5f605008     kernel32:KERNEL32.dll
 0002:0000000c       __imp__LocalAlloc@8        5f60500c     kernel32:KERNEL32.dll
 0002:00000010       __imp__LoadLibraryA@4      5f605010     kernel32:KERNEL32.dll
 0002:00000014       __imp__SetLastError@4      5f605014     kernel32:KERNEL32.dll
 0002:00000018       __imp__GetProcAddress@8    5f605018     kernel32:KERNEL32.dll
 0002:0000001c       __imp__InterlockedExchange@8 5f60501c     kernel32:KERNEL32.dll
 0002:00000020       __imp__RaiseException@16   5f605020     kernel32:KERNEL32.dll
 0002:00000024       __imp__GetLastError@0      5f605024     kernel32:KERNEL32.dll
 0002:00000028       \177KERNEL32_NULL_THUNK_DATA 5f605028     kernel32:KERNEL32.dll
 0002:0000002c       __imp_?Serialize@CObject@@UAEXAAVCArchive@@@Z 5f60502c     MFC42D:MFC42D.DLL
 0002:00000030       __imp_??0CObject@@IAE@XZ   5f605030     MFC42D:MFC42D.DLL
 0002:00000034       __imp_??4CString@@QAEABV0@PBD@Z 5f605034     MFC42D:MFC42D.DLL
 0002:00000038       __imp_?AfxGetModuleThreadState@@YGPAVAFX_MODULE_THREAD_STATE@@XZ 5f605038     MFC42D:MFC42D.DLL
 0002:0000003c       __imp_??3CNoTrackObject@@SGXPAX@Z 5f60503c     MFC42D:MFC42D.DLL
 0002:00000040       __imp_??1CObject@@UAE@XZ   5f605040     MFC42D:MFC42D.DLL
 0002:00000044       __imp_?GetValueAt@CMapPtrToPtr@@QBEPAXPAX@Z 5f605044     MFC42D:MFC42D.DLL
 0002:00000048       __imp_??3CObject@@SGXPAXPBDH@Z 5f605048     MFC42D:MFC42D.DLL
 0002:0000004c       __imp_?Lookup@CMapPtrToPtr@@QBEHPAXAAPAX@Z 5f60504c     MFC42D:MFC42D.DLL
 0002:00000050       __imp_?SetAt@CMapPtrToPtr@@QAEXPAX0@Z 5f605050     MFC42D:MFC42D.DLL
 0002:00000054       __imp_?FromHandlePermanent@CWnd@@SGPAV1@PAUHWND__@@@Z 5f605054     MFC42D:MFC42D.DLL
 0002:00000058       __imp_?AfxThrowResourceException@@YGXXZ 5f605058     MFC42D:MFC42D.DLL
 0002:0000005c       __imp_?AfxTrace@@YAXPBDZZ  5f60505c     MFC42D:MFC42D.DLL
 0002:00000060       __imp_?CreateEx@CWnd@@QAEHKPBD0KHHHHPAUHWND__@@PAUHMENU__@@PAX@Z 5f605060     MFC42D:MFC42D.DLL
 0002:00000064       __imp_?AfxRegisterWndClass@@YGPBDIPAUHICON__@@PAUHBRUSH__@@0@Z 5f605064     MFC42D:MFC42D.DLL
 0002:00000068       __imp_??2CObject@@SGPAXIPBDH@Z 5f605068     MFC42D:MFC42D.DLL
 0002:0000006c       __imp_?IsEmpty@CMapPtrToPtr@@QBEHXZ 5f60506c     MFC42D:MFC42D.DLL
 0002:00000070       __imp_?AfxEnableMemoryTracking@@YGHH@Z 5f605070     MFC42D:MFC42D.DLL
 0002:00000074       __imp_?RemoveHead@CPtrList@@QAEPAXXZ 5f605074     MFC42D:MFC42D.DLL
 0002:00000078       __imp_?IsEmpty@CPtrList@@QBEHXZ 5f605078     MFC42D:MFC42D.DLL
 0002:0000007c       __imp_?RemoveAll@CMapPtrToPtr@@QAEXXZ 5f60507c     MFC42D:MFC42D.DLL
 0002:00000080       __imp_?AfxAssertValidObject@@YGXPBVCObject@@PBDH@Z 5f605080     MFC42D:MFC42D.DLL
 0002:00000084       __imp_?RemoveKey@CMapPtrToPtr@@QAEHPAX@Z 5f605084     MFC42D:MFC42D.DLL
 0002:00000088       __imp_?AssertValid@CObject@@UBEXXZ 5f605088     MFC42D:MFC42D.DLL
 0002:0000008c       __imp_??6CDumpContext@@QAEAAV0@I@Z 5f60508c     MFC42D:MFC42D.DLL
 0002:00000090       __imp_??6CDumpContext@@QAEAAV0@PBD@Z 5f605090     MFC42D:MFC42D.DLL
 0002:00000094       __imp_?Dump@CObject@@UBEXAAVCDumpContext@@@Z 5f605094     MFC42D:MFC42D.DLL
 0002:00000098       __imp_?AddTail@CPtrList@@QAEPAU__POSITION@@PAX@Z 5f605098     MFC42D:MFC42D.DLL
 0002:0000009c       __imp_??2@YAPAXIPBDH@Z     5f60509c     MFC42D:MFC42D.DLL
 0002:000000a0       __imp_?Delete@CException@@QAEXXZ 5f6050a0     MFC42D:MFC42D.DLL
 0002:000000a4       __imp_?IsKindOf@CObject@@QBEHPBUCRuntimeClass@@@Z 5f6050a4     MFC42D:MFC42D.DLL
 0002:000000a8       __imp_?classCException@CException@@2UCRuntimeClass@@B 5f6050a8     MFC42D:MFC42D.DLL
 0002:000000ac       __imp_?AfxGetThread@@YGPAVCWinThread@@XZ 5f6050ac     MFC42D:MFC42D.DLL
 0002:000000b0       __imp_??6CDumpContext@@QAEAAV0@H@Z 5f6050b0     MFC42D:MFC42D.DLL
 0002:000000b4       __imp_??6CDumpContext@@QAEAAV0@PBX@Z 5f6050b4     MFC42D:MFC42D.DLL
 0002:000000b8       __imp_?GetBufferPtr@CFile@@UAEIIIPAPAX0@Z 5f6050b8     MFC42D:MFC42D.DLL
 0002:000000bc       __imp_?SetFilePath@CFile@@UAEXPBD@Z 5f6050bc     MFC42D:MFC42D.DLL
 0002:000000c0       __imp_?GetFilePath@CFile@@UBE?AVCString@@XZ 5f6050c0     MFC42D:MFC42D.DLL
 0002:000000c4       __imp_?GetFileTitle@CFile@@UBE?AVCString@@XZ 5f6050c4     MFC42D:MFC42D.DLL
 0002:000000c8       __imp_?GetFileName@CFile@@UBE?AVCString@@XZ 5f6050c8     MFC42D:MFC42D.DLL
 0002:000000cc       __imp_??1CFile@@UAE@XZ     5f6050cc     MFC42D:MFC42D.DLL
 0002:000000d0       __imp_??0CFile@@QAE@XZ     5f6050d0     MFC42D:MFC42D.DLL
 0002:000000d4       __imp_?AfxThrowFileException@@YGXHJPBD@Z 5f6050d4     MFC42D:MFC42D.DLL
 0002:000000d8       __imp_?AfxThrowNotSupportedException@@YGXXZ 5f6050d8     MFC42D:MFC42D.DLL
 0002:000000dc       __imp_?AssertValid@CFile@@UBEXXZ 5f6050dc     MFC42D:MFC42D.DLL
 0002:000000e0       __imp_??6CDumpContext@@QAEAAV0@PBVCObject@@@Z 5f6050e0     MFC42D:MFC42D.DLL
 0002:000000e4       __imp_?GetDepth@CDumpContext@@QBEHXZ 5f6050e4     MFC42D:MFC42D.DLL
 0002:000000e8       __imp_?Dump@CFile@@UBEXAAVCDumpContext@@@Z 5f6050e8     MFC42D:MFC42D.DLL
 0002:000000ec       __imp_?SetOccDialogInfo@CWnd@@MAEHPAU_AFX_OCC_DIALOG_INFO@@@Z 5f6050ec     MFC42D:MFC42D.DLL
 0002:000000f0       __imp_?IsFrameWnd@CWnd@@UBEHXZ 5f6050f0     MFC42D:MFC42D.DLL
 0002:000000f4       __imp_??3@YAXPAX@Z         5f6050f4     MFC42D:MFC42D.DLL
 0002:000000f8       __imp_??2@YAPAXI@Z         5f6050f8     MFC42D:MFC42D.DLL
 0002:000000fc       __imp_?PostNcDestroy@CWnd@@MAEXXZ 5f6050fc     MFC42D:MFC42D.DLL
 0002:00000100       __imp_?DefWindowProcA@CWnd@@MAEJIIJ@Z 5f605100     MFC42D:MFC42D.DLL
 0002:00000104       __imp_?OnWndMsg@CWnd@@MAEHIIJPAJ@Z 5f605104     MFC42D:MFC42D.DLL
 0002:00000108       __imp_?WindowProc@CWnd@@MAEJIIJ@Z 5f605108     MFC42D:MFC42D.DLL
 0002:0000010c       __imp_?OnAmbientProperty@CWnd@@UAEHPAVCOleControlSite@@JPAUtagVARIANT@@@Z 5f60510c     MFC42D:MFC42D.DLL
 0002:00000110       __imp_?PreTranslateMessage@CWnd@@UAEHPAUtagMSG@@@Z 5f605110     MFC42D:MFC42D.DLL
 0002:00000114       __imp_?EndModalState@CWnd@@UAEXXZ 5f605114     MFC42D:MFC42D.DLL
 0002:00000118       __imp_?BeginModalState@CWnd@@UAEXXZ 5f605118     MFC42D:MFC42D.DLL
 0002:0000011c       __imp_?AfxGetModuleState@@YGPAVAFX_MODULE_STATE@@XZ 5f60511c     MFC42D:MFC42D.DLL
 0002:00000120       __imp_?GetSuperWndProcAddr@CWnd@@MAEPAP6GJPAUHWND__@@IIJ@ZXZ 5f605120     MFC42D:MFC42D.DLL
 0002:00000124       __imp_?OnNotify@CWnd@@MAEHIJPAJ@Z 5f605124     MFC42D:MFC42D.DLL
 0002:00000128       __imp_?OnCommand@CWnd@@MAEHIJ@Z 5f605128     MFC42D:MFC42D.DLL
 0002:0000012c       __imp_?EndModalLoop@CWnd@@UAEXH@Z 5f60512c     MFC42D:MFC42D.DLL
 0002:00000130       __imp_?ContinueModal@CWnd@@UAEHXZ 5f605130     MFC42D:MFC42D.DLL
 0002:00000134       __imp_?WinHelpA@CWnd@@UAEXKI@Z 5f605134     MFC42D:MFC42D.DLL
 0002:00000138       __imp_?GetScrollBarCtrl@CWnd@@UBEPAVCScrollBar@@H@Z 5f605138     MFC42D:MFC42D.DLL
 0002:0000013c       __imp_?OnToolHitTest@CWnd@@UBEHVCPoint@@PAUtagTOOLINFOA@@@Z 5f60513c     MFC42D:MFC42D.DLL
 0002:00000140       __imp_?CalcWindowRect@CWnd@@UAEXPAUtagRECT@@I@Z 5f605140     MFC42D:MFC42D.DLL
 0002:00000144       __imp_?PreCreateWindow@CWnd@@UAEHAAUtagCREATESTRUCTA@@@Z 5f605144     MFC42D:MFC42D.DLL
 0002:00000148       __imp_?DestroyWindow@CWnd@@UAEHXZ 5f605148     MFC42D:MFC42D.DLL
 0002:0000014c       __imp_?Create@CWnd@@UAEHPBD0KABUtagRECT@@PAV1@IPAUCCreateContext@@@Z 5f60514c     MFC42D:MFC42D.DLL
 0002:00000150       __imp_?PreSubclassWindow@CWnd@@UAEXXZ 5f605150     MFC42D:MFC42D.DLL
 0002:00000154       __imp_?GetConnectionHook@CCmdTarget@@MAEPAUIConnectionPoint@@ABU_GUID@@@Z 5f605154     MFC42D:MFC42D.DLL
 0002:00000158       __imp_?GetExtraConnectionPoints@CCmdTarget@@MAEHPAVCPtrArray@@@Z 5f605158     MFC42D:MFC42D.DLL
 0002:0000015c       __imp_?GetInterfaceHook@CCmdTarget@@UAEPAUIUnknown@@PBX@Z 5f60515c     MFC42D:MFC42D.DLL
 0002:00000160       __imp_?OnCreateAggregates@CCmdTarget@@UAEHXZ 5f605160     MFC42D:MFC42D.DLL
 0002:00000164       __imp_?GetEventSinkMap@CCmdTarget@@MBEPBUAFX_EVENTSINKMAP@@XZ 5f605164     MFC42D:MFC42D.DLL
 0002:00000168       __imp_?GetInterfaceMap@CCmdTarget@@MBEPBUAFX_INTERFACEMAP@@XZ 5f605168     MFC42D:MFC42D.DLL
 0002:0000016c       __imp_?GetConnectionMap@CCmdTarget@@MBEPBUAFX_CONNECTIONMAP@@XZ 5f60516c     MFC42D:MFC42D.DLL
 0002:00000170       __imp_?GetDispatchMap@CCmdTarget@@MBEPBUAFX_DISPMAP@@XZ 5f605170     MFC42D:MFC42D.DLL
 0002:00000174       __imp_?GetCommandMap@CCmdTarget@@MBEPBUAFX_OLECMDMAP@@XZ 5f605174     MFC42D:MFC42D.DLL
 0002:00000178       __imp_?GetTypeLib@CCmdTarget@@UAEJKPAPAUITypeLib@@@Z 5f605178     MFC42D:MFC42D.DLL
 0002:0000017c       __imp_?GetTypeLibCache@CCmdTarget@@UAEPAVCTypeLibCache@@XZ 5f60517c     MFC42D:MFC42D.DLL
 0002:00000180       __imp_?GetTypeInfoCount@CCmdTarget@@UAEIXZ 5f605180     MFC42D:MFC42D.DLL
 0002:00000184       __imp_?GetDispatchIID@CCmdTarget@@UAEHPAU_GUID@@@Z 5f605184     MFC42D:MFC42D.DLL
 0002:00000188       __imp_?IsInvokeAllowed@CCmdTarget@@UAEHJ@Z 5f605188     MFC42D:MFC42D.DLL
 0002:0000018c       __imp_?OnFinalRelease@CWnd@@UAEXXZ 5f60518c     MFC42D:MFC42D.DLL
 0002:00000190       __imp_?OnCmdMsg@CCmdTarget@@UAEHIHPAXPAUAFX_CMDHANDLERINFO@@@Z 5f605190     MFC42D:MFC42D.DLL
 0002:00000194       __imp_?Dump@CWnd@@UBEXAAVCDumpContext@@@Z 5f605194     MFC42D:MFC42D.DLL
 0002:00000198       __imp_?AssertValid@CWnd@@UBEXXZ 5f605198     MFC42D:MFC42D.DLL
 0002:0000019c       __imp_?GetRuntimeClass@CWnd@@UBEPAUCRuntimeClass@@XZ 5f60519c     MFC42D:MFC42D.DLL
 0002:000001a0       __imp_??0CWnd@@QAE@XZ      5f6051a0     MFC42D:MFC42D.DLL
 0002:000001a4       __imp_??1CWnd@@UAE@XZ      5f6051a4     MFC42D:MFC42D.DLL
 0002:000001a8       __imp_?messageMap@CWnd@@1UAFX_MSGMAP@@B 5f6051a8     MFC42D:MFC42D.DLL
 0002:000001ac       __imp_?classCObject@CObject@@2UCRuntimeClass@@B 5f6051ac     MFC42D:MFC42D.DLL
 0002:000001b0       __imp_?classCFile@CFile@@2UCRuntimeClass@@B 5f6051b0     MFC42D:MFC42D.DLL
 0002:000001b4       __imp_??1CProcessLocalObject@@QAE@XZ 5f6051b4     MFC42D:MFC42D.DLL
 0002:000001b8       __imp_?GetData@CProcessLocalObject@@QAEPAVCNoTrackObject@@P6GPAV2@XZ@Z 5f6051b8     MFC42D:MFC42D.DLL
 0002:000001bc       __imp_??2CNoTrackObject@@SGPAXI@Z 5f6051bc     MFC42D:MFC42D.DLL
 0002:000001c0       __imp_?AfxGetAppModuleState@@YGPAVAFX_MODULE_STATE@@XZ 5f6051c0     MFC42D:MFC42D.DLL
 0002:000001c4       __imp_??3CObject@@SGXPAX@Z 5f6051c4     MFC42D:MFC42D.DLL
 0002:000001c8       __imp_?AfxInitExtensionModule@@YGHAAUAFX_EXTENSION_MODULE@@PAUHINSTANCE__@@@Z 5f6051c8     MFC42D:MFC42D.DLL
 0002:000001cc       __imp_?AfxAssertFailedLine@@YGHPBDH@Z 5f6051cc     MFC42D:MFC42D.DLL
 0002:000001d0       __imp_??2CObject@@SGPAXI@Z 5f6051d0     MFC42D:MFC42D.DLL
 0002:000001d4       __imp_??0CDynLinkLibrary@@QAE@AAUAFX_EXTENSION_MODULE@@H@Z 5f6051d4     MFC42D:MFC42D.DLL
 0002:000001d8       __imp_?AfxTermExtensionModule@@YGXAAUAFX_EXTENSION_MODULE@@H@Z 5f6051d8     MFC42D:MFC42D.DLL
 0002:000001dc       __imp_?AfxTermThread@@YGXPAUHINSTANCE__@@@Z 5f6051dc     MFC42D:MFC42D.DLL
 0002:000001e0       __imp_?OnChildNotify@CWnd@@MAEHIIJPAJ@Z 5f6051e0     MFC42D:MFC42D.DLL
 0002:000001e4       __imp_?CheckAutoCenter@CWnd@@UAEHXZ 5f6051e4     MFC42D:MFC42D.DLL
 0002:000001e8       __imp_?DoDataExchange@CWnd@@MAEXPAVCDataExchange@@@Z 5f6051e8     MFC42D:MFC42D.DLL
 0002:000001ec       \177MFC42D_NULL_THUNK_DATA 5f6051ec     MFC42D:MFC42D.DLL
 0002:000001f0       __imp___adjust_fdiv        5f6051f0     msvcrtd:MSVCRTD.dll
 0002:000001f4       __imp___malloc_dbg         5f6051f4     msvcrtd:MSVCRTD.dll
 0002:000001f8       __imp___initterm           5f6051f8     msvcrtd:MSVCRTD.dll
 0002:000001fc       __imp___free_dbg           5f6051fc     msvcrtd:MSVCRTD.dll
 0002:00000200       __imp___onexit             5f605200     msvcrtd:MSVCRTD.dll
 0002:00000204       __imp____dllonexit         5f605204     msvcrtd:MSVCRTD.dll
 0002:00000208       __imp_??1type_info@@UAE@XZ 5f605208     msvcrtd:MSVCRTD.dll
 0002:0000020c       __imp____CxxFrameHandler   5f60520c     msvcrtd:MSVCRTD.dll
 0002:00000210       __imp_?terminate@@YAXXZ    5f605210     msvcrtd:MSVCRTD.dll
 0002:00000214       __imp__memset              5f605214     msvcrtd:MSVCRTD.dll
 0002:00000218       __imp___except_handler3    5f605218     msvcrtd:MSVCRTD.dll
 0002:0000021c       \177MSVCRTD_NULL_THUNK_DATA 5f60521c     msvcrtd:MSVCRTD.dll
 0002:00000220       __imp__PostMessageA@16     5f605220     user32:USER32.dll
 0002:00000224       __imp__KillTimer@8         5f605224     user32:USER32.dll
 0002:00000228       __imp__PeekMessageA@20     5f605228     user32:USER32.dll
 0002:0000022c       __imp__WaitMessage@0       5f60522c     user32:USER32.dll
 0002:00000230       __imp__SetTimer@16         5f605230     user32:USER32.dll
 0002:00000234       __imp__DispatchMessageA@4  5f605234     user32:USER32.dll
 0002:00000238       \177USER32_NULL_THUNK_DATA 5f605238     user32:USER32.dll
 0002:00000260       _IID_IDocHostUIHandlerDispatch 5f605260     dllnet.obj
 0002:00000270       _IID_IInternalConnection   5f605270     dllnet.obj
 0002:00000280       _IID_IAxWinAmbientDispatch 5f605280     dllnet.obj
 0002:00000290       _IID_IAxWinHostWindow      5f605290     dllnet.obj
 0002:000002a0       _IID_IRegistrar            5f6052a0     dllnet.obj
 0002:000002b0       _CLSID_Registrar           5f6052b0     dllnet.obj
 0002:000002c0       _LIBID_ATLLib              5f6052c0     dllnet.obj
 0002:000002d0       ??_C@_0L@LDKI@MFC42D?4DLL?$AA@ 5f6052d0     dllnet.obj
 0002:000002e0       ?classCSocketFile@CSocketFile@@2UCRuntimeClass@@B 5f6052e0     sockcore.obj
 0002:000002f8       ??_C@_0M@FJKI@CSocketFile?$AA@ 5f6052f8     sockcore.obj
 0002:00000308       ?classCSocket@CSocket@@2UCRuntimeClass@@B 5f605308     sockcore.obj
 0002:00000320       ??_C@_07MBCI@CSocket?$AA@  5f605320     sockcore.obj
 0002:00000328       ?classCAsyncSocket@CAsyncSocket@@2UCRuntimeClass@@B 5f605328     sockcore.obj
 0002:00000340       ??_C@_0N@CCKH@CAsyncSocket?$AA@ 5f605340     sockcore.obj
 0002:00000350       ?messageMap@CSocketWnd@@1UAFX_MSGMAP@@B 5f605350     sockcore.obj
 0002:00000358       ?_messageEntries@CSocketWnd@@0QBUAFX_MSGMAP_ENTRY@@B 5f605358     sockcore.obj
 0002:000003a4       ??_7_AFX_SOCK_STATE@@6B@   5f6053a4     sockcore.obj
 0002:000003ac       ??_7CAsyncSocket@@6B@      5f6053ac     sockcore.obj
 0002:000003f8       ??_7CNoTrackObject@@6B@    5f6053f8     sockcore.obj
 0002:000003fc       ??_C@_02DILL@?$CFs?$AA@    5f6053fc     sockcore.obj
 0002:00000400       ??_C@_0DB@FJKP@Warning?3?5unable?5to?5create?5socket@ 5f605400     sockcore.obj
 0002:00000434       ??_C@_0BJ@HDPG@Socket?5Notification?5Sink?$AA@ 5f605434     sockcore.obj
 0002:00000450       ??_C@_01BJG@?6?$AA@        5f605450     sockcore.obj
 0002:00000454       ??_C@_0BA@MMD@INVALID_SOCKET?6?$AA@ 5f605454     sockcore.obj
 0002:00000464       ??_C@_0N@HJN@m_hSocket?5?$DN?5?$AA@ 5f605464     sockcore.obj
 0002:00000478       ??_7CSocket@@6B@           5f605478     sockcore.obj
 0002:000004c8       ??_C@_0DG@NLAD@Error?3?5caught?5exception?5in?5PumpM@ 5f6054c8     sockcore.obj
 0002:00000500       ??_C@_0BD@MNOG@m_nConnectError?5?$DN?5?$AA@ 5f605500     sockcore.obj
 0002:00000514       ??_C@_0BA@EKGE@m_pbBlocking?5?$DN?5?$AA@ 5f605514     sockcore.obj
 0002:00000528       ??_7CSocketFile@@6B@       5f605528     sockcore.obj
 0002:00000584       ??_C@_0DB@HFNB@Warning?5?9?5Attempt?5made?5to?5seek?5o@ 5f605584     sockcore.obj
 0002:000005b8       ??_C@_0O@FJPJ@with?5socket?3?5?$AA@ 5f6055b8     sockcore.obj
 0002:000005c8       ??_C@_0BA@JPDC@with?5no?5socket?6?$AA@ 5f6055c8     sockcore.obj
 0002:000005dc       ??_7CSocketWnd@@6B@        5f6055dc     sockcore.obj
 0002:0000069c       ??_C@_0CH@KFAI@E?3?28168?2vc98?2mfc?2mfc?2include?2afx@ 5f60569c     sockcore.obj
 0002:000006f8       ??_7type_info@@6B@         5f6056f8     msvcrtd:ti_inst.obj
 0002:000006fc       ??_C@_08JKC@crtdll?4c?$AA@ 5f6056fc     msvcrtd:crtdll.obj
 0002:00000710       __sz_WSOCK32               5f605710     wsock32:WSOCK32.dll
 0002:00000720       ??_R1A@?0A@A@CNoTrackObject@@8 5f605720     sockcore.obj
 0002:00000738       ??_R1A@?0A@A@_AFX_SOCK_STATE@@8 5f605738     sockcore.obj
 0002:00000750       ??_R2_AFX_SOCK_STATE@@8    5f605750     sockcore.obj
 0002:00000760       ??_R3_AFX_SOCK_STATE@@8    5f605760     sockcore.obj
 0002:00000770       ??_R4_AFX_SOCK_STATE@@6B@  5f605770     sockcore.obj
 0002:00000788       ??_R1A@?0A@A@CObject@@8    5f605788     sockcore.obj
 0002:000007a0       ??_R1A@?0A@A@CAsyncSocket@@8 5f6057a0     sockcore.obj
 0002:000007b8       ??_R2CAsyncSocket@@8       5f6057b8     sockcore.obj
 0002:000007c8       ??_R3CAsyncSocket@@8       5f6057c8     sockcore.obj
 0002:000007d8       ??_R4CAsyncSocket@@6B@     5f6057d8     sockcore.obj
 0002:000007ec       ??_R2CNoTrackObject@@8     5f6057ec     sockcore.obj
 0002:000007f8       ??_R3CNoTrackObject@@8     5f6057f8     sockcore.obj
 0002:00000808       ??_R4CNoTrackObject@@6B@   5f605808     sockcore.obj
 0002:00000820       ??_R1A@?0A@A@CSocket@@8    5f605820     sockcore.obj
 0002:00000838       ??_R2CSocket@@8            5f605838     sockcore.obj
 0002:00000848       ??_R3CSocket@@8            5f605848     sockcore.obj
 0002:00000858       ??_R4CSocket@@6B@          5f605858     sockcore.obj
 0002:00000870       ??_R1A@?0A@A@CFile@@8      5f605870     sockcore.obj
 0002:00000888       ??_R1A@?0A@A@CSocketFile@@8 5f605888     sockcore.obj
 0002:000008a0       ??_R2CSocketFile@@8        5f6058a0     sockcore.obj
 0002:000008b0       ??_R3CSocketFile@@8        5f6058b0     sockcore.obj
 0002:000008c0       ??_R4CSocketFile@@6B@      5f6058c0     sockcore.obj
 0002:000008d8       ??_R1A@?0A@A@CCmdTarget@@8 5f6058d8     sockcore.obj
 0002:000008f0       ??_R1A@?0A@A@CWnd@@8       5f6058f0     sockcore.obj
 0002:00000908       ??_R1A@?0A@A@CSocketWnd@@8 5f605908     sockcore.obj
 0002:00000920       ??_R2CSocketWnd@@8         5f605920     sockcore.obj
 0002:00000938       ??_R3CSocketWnd@@8         5f605938     sockcore.obj
 0002:00000948       ??_R4CSocketWnd@@6B@       5f605948     sockcore.obj
 0002:00000960       ??_R1A@?0A@A@type_info@@8  5f605960     msvcrtd:ti_inst.obj
 0002:00000978       ??_R2type_info@@8          5f605978     msvcrtd:ti_inst.obj
 0002:00000980       ??_R3type_info@@8          5f605980     msvcrtd:ti_inst.obj
 0002:00000990       ??_R4type_info@@6B@        5f605990     msvcrtd:ti_inst.obj
 0002:00000b48       __DELAY_IMPORT_DESCRIPTOR_WSOCK32 5f605b48     wsock32:WSOCK32.dll
 0002:00000b68       __NULL_DELAY_IMPORT_DESCRIPTOR 5f605b68     wsock32:WSOCK32.dll
 0002:00000bf4       \177WSOCK32_NULL_THUNK_DATA_DLN 5f605bf4     wsock32:WSOCK32.dll
 0002:00000bfc       \177WSOCK32_NULL_THUNK_DATA_DLB 5f605bfc     wsock32:WSOCK32.dll
 0002:00000c68       __IMPORT_DESCRIPTOR_MFC42D 5f605c68     MFC42D:MFC42D.DLL
 0002:00000c7c       __IMPORT_DESCRIPTOR_MSVCRTD 5f605c7c     msvcrtd:MSVCRTD.dll
 0002:00000c90       __IMPORT_DESCRIPTOR_KERNEL32 5f605c90     kernel32:KERNEL32.dll
 0002:00000ca4       __IMPORT_DESCRIPTOR_USER32 5f605ca4     user32:USER32.dll
 0002:00000cb8       __NULL_IMPORT_DESCRIPTOR   5f605cb8     MFC42D:MFC42D.DLL
 0003:00000000       ___xc_a                    5f607000     msvcrtd:cinitexe.obj
 0003:00000008       ___xc_z                    5f607008     msvcrtd:cinitexe.obj
 0003:0000000c       ___xi_a                    5f60700c     msvcrtd:cinitexe.obj
 0003:00000010       ___xi_z                    5f607010     msvcrtd:cinitexe.obj
 0003:0000002c       __pRawDllMain              5f60702c     dllnet.obj
 0003:00000030       ?_afxForceVectorDelete_mfcn@@3P6AXXZA 5f607030     dllnet.obj
 0003:00000038       ?GUID_ATLVer30@ATL@@3U_GUID@@A 5f607038     dllnet.obj
 0003:00000068       ??_R0?AVCNoTrackObject@@@8 5f607068     sockcore.obj
 0003:00000088       ??_R0?AV_AFX_SOCK_STATE@@@8 5f607088     sockcore.obj
 0003:000000a8       ??_R0?AVCObject@@@8        5f6070a8     sockcore.obj
 0003:000000c0       ??_R0?AVCAsyncSocket@@@8   5f6070c0     sockcore.obj
 0003:000000e0       ??_R0?AVCSocket@@@8        5f6070e0     sockcore.obj
 0003:000000f8       ??_R0PAVCException@@@8     5f6070f8     sockcore.obj
 0003:00000118       ??_R0?AVCFile@@@8          5f607118     sockcore.obj
 0003:00000130       ??_R0?AVCSocketFile@@@8    5f607130     sockcore.obj
 0003:00000150       ??_R0?AVCCmdTarget@@@8     5f607150     sockcore.obj
 0003:00000170       ??_R0?AVCWnd@@@8           5f607170     sockcore.obj
 0003:00000188       ??_R0?AVCSocketWnd@@@8     5f607188     sockcore.obj
 0003:000001b0       ??_R0?AVtype_info@@@8      5f6071b0     msvcrtd:ti_inst.obj
 0003:000001c8       __imp__WSAAsyncSelect@16   5f6071c8     wsock32:WSOCK32.dll
 0003:000001cc       __imp__WSAStartup@8        5f6071cc     wsock32:WSOCK32.dll
 0003:000001d0       __imp__WSASetLastError@4   5f6071d0     wsock32:WSOCK32.dll
 0003:000001d4       __imp__inet_ntoa@4         5f6071d4     wsock32:WSOCK32.dll
 0003:000001d8       __imp__ntohs@4             5f6071d8     wsock32:WSOCK32.dll
 0003:000001dc       __imp__accept@12           5f6071dc     wsock32:WSOCK32.dll
 0003:000001e0       __imp__htons@4             5f6071e0     wsock32:WSOCK32.dll
 0003:000001e4       __imp__inet_addr@4         5f6071e4     wsock32:WSOCK32.dll
 0003:000001e8       __imp__htonl@4             5f6071e8     wsock32:WSOCK32.dll
 0003:000001ec       __imp__closesocket@4       5f6071ec     wsock32:WSOCK32.dll
 0003:000001f0       __imp__gethostbyname@4     5f6071f0     wsock32:WSOCK32.dll
 0003:000001f4       __imp__recv@16             5f6071f4     wsock32:WSOCK32.dll
 0003:000001f8       __imp__send@16             5f6071f8     wsock32:WSOCK32.dll
 0003:000001fc       __imp__WSACleanup@0        5f6071fc     wsock32:WSOCK32.dll
 0003:00000200       __imp__WSAGetLastError@0   5f607200     wsock32:WSOCK32.dll
 0003:00000204       __imp__socket@12           5f607204     wsock32:WSOCK32.dll
 0003:00000208       __imp__recvfrom@24         5f607208     wsock32:WSOCK32.dll
 0003:0000020c       __imp__sendto@24           5f60720c     wsock32:WSOCK32.dll
 0003:00000210       __imp__connect@12          5f607210     wsock32:WSOCK32.dll
 0003:00000214       __imp__getpeername@12      5f607214     wsock32:WSOCK32.dll
 0003:00000218       __imp__getsockname@12      5f607218     wsock32:WSOCK32.dll
 0003:0000021c       __imp__setsockopt@20       5f60721c     wsock32:WSOCK32.dll
 0003:00000220       __imp__getsockopt@20       5f607220     wsock32:WSOCK32.dll
 0003:00000224       __imp__bind@12             5f607224     wsock32:WSOCK32.dll
 0003:00000228       __imp__ioctlsocket@12      5f607228     wsock32:WSOCK32.dll
 0003:0000022c       __imp__listen@8            5f60722c     wsock32:WSOCK32.dll
 0003:00000230       __imp__shutdown@8          5f607230     wsock32:WSOCK32.dll
 0003:00000234       \177WSOCK32_NULL_THUNK_DATA_DLA 5f607234     wsock32:WSOCK32.dll
 0003:00000238       ?ATL_CREATE_OBJECT@CComApartment@ATL@@2IA 5f607238     dllnet.obj
 0003:00000240       ?m_libid@CComModule@ATL@@2U_GUID@@A 5f607240     dllnet.obj
 0003:00000250       ?_pModule@ATL@@3PAVCComModule@1@A 5f607250     dllnet.obj
 0003:0000026c       ?_afxSockState@@3V?$CProcessLocal@V_AFX_SOCK_STATE@@@@A 5f60726c     sockcore.obj
 0003:00000274       __hmod__WSOCK32            5f607274     wsock32:WSOCK32.dll
 0003:00000278       ___puiHead                 5f607278     delayimp:delayhlp.obj
 0003:0000027c       ___pfnDliFailureHook       5f60727c     delayimp:delayhk1.obj
 0003:00000280       ___pfnDliNotifyHook        5f607280     delayimp:delayhk2.obj
 0003:00000284       __adjust_fdiv              5f607284     <common>
 0003:00000288       ___onexitend               5f607288     <common>
 0003:0000028c       ___onexitbegin             5f60728c     <common>

 entry point at        0001:000006e0

 Static symbols

 0001:00000f6e       _$E375                     5f601f6e f   sockcore.obj
 0001:00000f7d       _$E372                     5f601f7d f   sockcore.obj
 0001:00000f82       _$E374                     5f601f82 f   sockcore.obj
 0001:00000f94       _$E373                     5f601f94 f   sockcore.obj
 0001:00003330       ?_AfxForceVectorDelete@@YAXXZ 5f604330 f   dllnet.obj
 0001:000004d0       ?ArrayUnwindFilter@@YAHPAU_EXCEPTION_POINTERS@@@Z 5f6014d0 f   msvcrtd:ehvecdtr.obj
 0001:00000cc3       ?OverlayIAT@@YGXPAU_IMAGE_THUNK_DATA32@@PBU1@@Z 5f601cc3 f   delayimp:delayhlp.obj

 33 bytes saved through ICF

